:100000008A110A1205280000090083160E309F008D
:10001000810164308F00831241309F0083162130AC
:100020008500FE308600831286018501BC01BD017A
:10003000BE01BF01C001C101C201C301C401C501AC
:10004000C701C801C901CA01CB01CC0106142C307B
:10005000A0000130A100CB2206102C30A0000130FE
:10006000A100CB2206142C30A0000130A100CB222D
:10007000061051214608033C031D772837213A0812
:10008000A0003B08A100A3010030A922031D4928BC
:1000900075281F3083050130AC00AD012C08A0008D
:1000A0002D08A1003B08A3003A08B822031D6E28C2
:1000B00006142C30A0000130A100CB2206102C30F9
:1000C000A0000130A100CB220130AC0700300318A2
:1000D000013E03186E28AD07031C4E281F30830510
:1000E000F430A0000130A100CB2251213A281F306A
:1000F00083054608063C031D9428372106143C0856
:100100003A07BC003D080318013E3B07BD00203004
:10011000A0000330A100CB2206102030A000033045
:10012000A100CB22512179281F3083054608073CC6
:10013000031DB128372106143E083A07BE003F08C8
:100140000318013E3B07BF002030A0000330A10090
:10015000CB2206102030A0000330A100CB22512179
:1001600096281F30830546080B3C031DCE283721F7
:10017000061440083A07C00041080318013E3B0737
:10018000C1002030A0000330A100CB220610203097
:10019000A0000330A100CB225121B3281F308305DA
:1001A00046080C3C031DEB283721061442083A0789
:1001B000C20043080318013E3B07C3002030A000E3
:1001C0000330A100CB2206102030A0000330A10094
:1001D000CB225121D0281F3083054608143C031D33
:1001E00008293721061444083A07C40045080318B3
:1001F000013E3B07C5002030A0000330A100CB2208
:1002000006102030A0000330A100CB225121ED28A0
:100210001F308305861B33294408A0004508A10030
:10022000A3010030A922031D162935291F3083059B
:100230000130B000B1013008A0003108A10045082C
:10024000A3004408B822031D3129A6211922013038
:10025000B00700300318013E03183129B107031C11
:100260001B291F3083051F308305392836291F14A9
:1002700083169F171F1300308312A000FE228316DF
:100280001E088312BA001E08BB003A08A0003B08F3
:10029000A1006430A200A3018D22BA002108BB0096
:1002A0000800061956290130C70059291F30830557
:1002B000C7011F308305861960290230C8006329F1
:1002C0001F308305C8011F308305061A6A290530CF
:1002D000C9006D291F308305C9011F308305861AA7
:1002E00074290A30CA0077291F308305CA011F30DC
:1002F0008305061B7E291430CB0081291F3083051E
:10030000CB011F30830547084807CE0000010318C2
:10031000013E003ECF004E084907CE004F080318AB
:10032000013E003ECF004E084A07CE004F0803189A
:10033000013E003ECF004E084B07CE004F08031889
:10034000013E003ECF004E08C60008003C08A00059
:100350003D08A100A3010030A922031DB029D22924
:100360001F3083050130AC00AD012C08A0002D0822
:10037000A1003D08A3003C08B822031DD029851424
:100380000614E830A0000330A100CB220130AC07F6
:1003900000300318013E0318D029AD07031CB5290E
:1003A0001F3083053E08A0003F08A100A3010030D4
:1003B000A922031DDC29162A1F3083050130AC0059
:1003C000AD012C08A0002D08A1003F08A3003E08A5
:1003D000B822031D142A851406140130AE00AF01A3
:1003E0002E08A0002F08A100A3013C30B822031D55
:1003F000082AE830A0000330A100CB220130AE076C
:1004000000300318013E0318082AAF07031CF02927
:100410001F3083050130AC0700300318013E03187C
:10042000142AAD07031CE1291F308305851006102F
:1004300008004008A0004108A100A3010030A92243
:10044000031D232A452A1F3083050130AC00AD016E
:100450002C08A0002D08A1004108A3004008B822E4
:10046000031D432A85100610E830A0000330A100C8
:10047000CB220130AC0700300318013E0318432A99
:10048000AD07031C282A1F3083054208A00043083B
:10049000A100A3010030A922031D4F2A892A1F3081
:1004A00083050130AC00AD012C08A0002D08A1008F
:1004B0004308A3004208B822031D872A85100610AE
:1004C0000130AE00AF012E08A0002F08A100A3014B
:1004D0003C30B822031D7B2AE830A0000330A10085
:1004E000CB220130AE0700300318013E03187B2AEF
:1004F000AF07031C632A1F3083050130AC070030AF
:100500000318013E0318872AAD07031C542A1F3025
:1005100083058510061008008C2A1030A600A5015E
:10052000A401210DA40DA50D2208A4022308031C7B
:10053000230FA5020318A32A2208A40723080318DF
:10054000230FA5070310A00DA10DA60B912A2008CB
:100550000800A2000530BB2AA2000230BB2AA2007C
:100560000630BB2AA2000330BB2AA2000430BB2AFB
:10057000A2000130BB2AA80023082102031DC22AC1
:100580002208200204300318013003190230280524
:10059000031DFF300800A0080319D62ADD22A0039E
:1005A00000000000000000000000CB2AA108031991
:1005B0000800DD22A103A003CB2A0C30A500A50B67
:1005C000DF2A000000001230A200A20BEC2AEE226B
:1005D000EE22000000000800EE22E52A0D30A40003
:1005E000A40BF02A000008000A30A802031C08002F
:1005F000F92A0630A802031C0800F92AA00DA00D54
:10060000A00D3830A005C13020049F001430A80090
:0E061000F4221F151F190A2B0C131F100800CF
:02400E00702F11
:00000001FF
